:020000040000FA
:06000000BCEF18F0120035
:0600080055EF11F012009B
:06001800B2EF11F012002E
:06102A000200A9310000E4
:10103000AB00000010000000A4310000C50000005B
:0410400005000000A7
:0C104400D9CFE6FFE1CFD9FFE652A09A19
:101050006A6A686A706A010EE66EE66AE66A710E8E
:10106000E66E0F0EE66E8AEC18F00B6E050EE15E72
:101070000B50160E6F6E9F0E6B6E7B0E696EDF6AE5
:10108000DF500B6E0C6A080E0B5C000E0C5810E261
:10109000DF50040DF3CFE9FFF4CFEAFF000EE9269D
:1010A000040EEA22EE6AEE6AEE6AEE6ADF2AE8D7FA
:1010B0006D8C6E6A6D986D9C68A607D0689600016D
:1010C000736B786B796B7A6BF7D70001010E8A6FBF
:1010D0008B6F8C6B8D6B806BDF6A020EDF5C26E2A0
:1010E000EA6ADF34FE0BEA36E96E6B0EE926000E83
:1010F000EA22EE6AED6AEA6ADF34FE0BEA36E96E4E
:10110000670EE926000EEA22EE6AED6ADF50EA6A0F
:10111000840FE96E000EEA22EF6ADF50EA6A860F5A
:10112000E96E000EEA22EF6ADF2AD7D70001080E27
:101130006B6F040E6C6F160E706E0401200E026F42
:10114000040E036F080E016F840E006F0001616BC7
:10115000606BE552E552E7CFD9FF1200D9CFE6FF29
:10116000E1CFD9FFE6520001600507E16DBA05D075
:10117000686A69806988020E606F6850040B06E037
:101180006950040B03E0689494EC0EF06DB259D0F2
:101190006850010B09E06950010B06E053DFA08A9B
:1011A0000001040E606F68906850100B06E06950F3
:1011B000100B03E07FEC0EF0689868AC19D069ACB6
:1011C0000FD0010EE66EE66A000EE66EE66A730E5A
:1011D000E66EE66A42EC17F00B6E060EE15E0B500F
:1011E000689C0001885101E08807885101E1FBD922
:1011F0006850200B05E06950200B02E066EC0EF011
:101200006850020B13E06950020B10E0010EE66E0D
:10121000E66A000EE66EE66AE6687F0EE66E42EC6F
:1012200017F00B6E060EE15E0B506A6A040E0001A9
:10123000E76E6019E8AE02D0E73402D0E750605D97
:1012400002E2A19A39D069A636D0DF6A040EDF5CCB
:1012500032E268A630D06CCF81F000018151780B6A
:10126000E842E842E842826F689681B506D0825132
:10127000EA6A860FE96E000E05D08251EA6A840F91
:10128000E96E000EEA22EF70825103E1ABEC0EF042
:1012900010D0000EE66EE66A810EE66E000EE66E77
:1012A000720EE66EE66A42EC17F00B6E060EE15E19
:1012B0000B50DF2ACBD7A19AE552E552E7CFD9FFF1
:1012C0001200D9CFE6FFE1CFD9FF020EE126FD0ED5
:1012D000DBA407D0E66AFE0EDBCFE6FF13DAE552A9
:1012E000E552FD0EDBA208D0010EE66EFE0EDBCF4E
:1012F000E6FF08DAE552E552FE0EDB500C6A700F8D
:101300000B6E0F0E0C220BC0DEFF0CC0DDFFDECF1C
:10131000E9FFDDCFEAFFFD0EDBCFEFFF020EE15C60
:1013200002E2E16AE552E16EE552E7CFD9FF120031
:10133000D9CFE6FFE1CFD9FF020EE126FD0EDB504B
:101340000AE0FE0EEA6ADB34FE0BEA36E96E6B0E4B
:10135000E926000E09D0FE0EEA6ADB34FE0BEA36FF
:10136000E96E670EE926000EEA22EECFDEFFEDCF32
:10137000DDFFD9CFE9FFDACFEAFFEE50ED1003E150
:10138000F36AF46A44D0DECFE9FFDDCFEAFF020E54
:10139000E926000EEA22FB0EDBCFEEFFFC0EDBCFD0
:1013A000EDFFDECFE9FFDDCFEAFFEE52FA0EDBCF35
:1013B000EFFF400EDECFE9FFDDCFEAFFE850EF168A
:1013C000880EDECFE9FFDDCFEAFFE850EF12FD0E19
:1013D000DB500AE0FE0EEA6ADB34FE0BEA36E96E09
:1013E0006B0EE926000E09D0FE0EEA6ADB34FE0B16
:1013F000EA36E96E670EE926000EEA22EF74DECFC8
:101400000BF0DDCF0CF00BC0F3FF0CC0F4FF020EAD
:10141000E15C02E2E16AE552E16EE552E7CFD9FF15
:101420001200D9CFE6FFE1CFD9FF020EE126FE0E72
:10143000DB5020E165C0E9FF66C0EAFFEE52080E0E
:10144000EF6E65C0E9FF66C0EAFF020EE926000EF6
:10145000EA22200EEE6E040EED6E65C0E9FF66C056
:10146000EAFF8C0EEF6E6BC0E9FF6CC0EAFF840EE2
:10147000EF6E3BD0FD0EDB50E8240D6EFE0EDB5010
:10148000040DF3500D24040DF3CF0BF0F4CF0CF04A
:10149000000E0B26040E0C220BC0DEFF0CC0DDFF7D
:1014A000840EDECFE9FFDDCFEAFFE850EF12FD0E3C
:1014B000DB50E8240D6EFE0EDB50040DF3500D24BE
:1014C000010F040DF3CF0BF0F4CF0CF0000E0B2640
:1014D000040E0C220BC0DEFF0CC0DDFF840EDECF3D
:1014E000E9FFDDCFEAFFE850EF12020EE15C02E215
:1014F000E16AE552E16EE552E7CFD9FF1200D9CF9C
:10150000E6FFE1CFD9FF6DA84ED0FE0EEA6ADB34CC
:10151000FE0BEA36E96E6B0EE926000EEA22EE506B
:10152000EFCFEAFFE96E400EEE16EE6AEE6AEE6A63
:10153000FE0EEA6ADB34FE0BEA36E96E6B0EE92634
:10154000000EEA22EE50EFCFEAFFE96EEE7CFE0ECF
:10155000EA6ADB34FE0BEA36E96E6B0EE926000E12
:10156000EA22EF74400E0B6EFE0EEA6ADB34FE0BCD
:10157000EA36E96E6B0EE926000EEA22EE50EFCF56
:10158000EAFFE96E0B50EF16FE0EEA6ADB34FE0B43
:10159000EA36E96E6B0EE926000EEA22EE50EFCF36
:1015A000EAFFE96EEF7CE552E7CFD9FF12006D6AE2
:1015B000696A0001606B12000001605113E16D6AFD
:1015C000696A160E6F6E9F0E6B6E7B0E696ED08E03
:1015D000A28AA08AF28E6DB602D06D86FCD7000179
:1015E000010E606F120000018A514DE1010E8A6FF9
:1015F0008B5149E1010E8B6F020E705D0DE16BC0E6
:10160000E9FF6CC0EAFFEE52EF6A6BC0E9FF6CC005
:10161000EAFFC80EEF6E1200700535E1836B63C000
:10162000E9FF64C0EAFFEE52080EEF6E63C0E9FF07
:1016300064C0EAFF020EE926000EEA22200EEE6EDA
:10164000040EED6E63C0E9FF64C0EAFF840EEF6E26
:10165000010E836F65C0E9FF66C0EAFFEE52080E17
:10166000EF6E65C0E9FF66C0EAFF020EE926000ED4
:10167000EA22200EEE6E040EED6E65C0E9FF66C034
:10168000EAFF800EEF6E120000018C6B8D6B020E74
:10169000705D18E165C0E9FF66C0EAFFEE52080E12
:1016A000EF6E65C0E9FF66C0EAFF020EE926000E94
:1016B000EA22280EEE6E040EED6E65C0E9FF66C0EC
:1016C000EAFF1DD074510401265D0001755104012B
:1016D000275904E226C474F027C475F0CAD86BC039
:1016E000E9FF6CC0EAFF020EE926000EEA22280E8E
:1016F000EE6E040EED6E6BC0E9FF6CC0EAFFC80E23
:10170000EF6E1200D9CFE6FFE1CFD9FF020EE1263E
:10171000000EDE6E040EDD6EFD0EDB50E8240D6E55
:10172000FE0EDB50040DF3500D24040DF4CF0CF02D
:10173000D9CFE9FFDACFEAFFF350EE260C50ED22C5
:10174000DECFE9FFDDCFEAFFEF9EFD0EDB500AE1C1
:10175000FE0EEA6ADB34FE0BEA36E96E670EE92616
:10176000000E09D0FE0EEA6ADB34FE0BEA36E96EA3
:101770006B0EE926000EEA22DECFEEFFDDCFEDFF95
:10178000DECFE9FFDDCFEAFFEF9CDECFE9FFDDCF63
:10179000EAFF040EE926000EEA22EF8C020EE15C5D
:1017A00002E2E16AE552E16EE552E7CFD9FF1200AD
:1017B0006D98000173BF2BD078AF09D0020E706F07
:1017C0008D5101E161DF00018B6B8A6B120065C0F6
:1017D000E9FF66C0EAFFEE52080EEF6E65C0E9FF52
:1017E00066C0EAFF020EE926000EEA22200EEE6E27
:1017F000040EED6E65C0E9FF66C0EAFF8C0EEF6E69
:101800006BC0E9FF6CC0EAFF840EEF6E12000401AA
:1018100020AF0DD00001010E706F8C5101E134DF5B
:1018200000018B6B8A6B895123E1F3EF0AF0000111
:10183000020E706F65C0E9FF66C0EAFFEE52080E47
:10184000EF6E65C0E9FF66C0EAFF020EE926000EF2
:10185000EA22200EEE6E040EED6E65C0E9FF66C052
:10186000EAFF840EEF6E8B6B8A6B895101E1BBDE60
:101870001200D9CFE6FFE1CFD9FFE652080EDF6EA6
:101880000001745D000E75590AE274C0DFFF6F51EC
:1018900002E1010E03D06F0502E1020E6F6FDF500F
:1018A0000C6AE850745D746F0C507559756F6BC09D
:1018B000E9FF6CC0EAFFEE52DFCFEFFF280E7D6F2D
:1018C000040E7E6F73B118D0DF502DE071C0F6FFAB
:1018D00072C0F7FF712B000E72230800F550E66E00
:1018E0007DC0E9FF7EC0EAFF7D2B000E7E23E5521E
:1018F000E750EF6EDF06E8D7DF5015E071C0E9FF73
:1019000072C0EAFF712B000E7223EF50E66E7DC0AD
:10191000E9FF7EC0EAFF7D2B000E7E23E552E750F3
:10192000EF6EDF06E9D7E552E552E7CFD9FF1200A7
:10193000D9CFE6FFE1CFD9FF020EE12663C0E9FF70
:1019400064C0EAFFEE52EFCFDFFFDFCF0BF00B50AA
:101950000001795D000E7A5902E279C0DFFFDF50A5
:101960000B6E0C6AE850795D796F0C507A597A6F7A
:10197000010EDB6ADF50F36E010EDBCFF4FFF35094
:10198000F45C16E2010EDB50EA6A280FE96E040EE1
:10199000EA22EF50E66E76C0E9FF77C0EAFF762BC9
:1019A000000E7723E552E750EF6E010EDB2AE2D7F7
:1019B000000ED8807955000E7A5527E265C0E9FF00
:1019C00066C0EAFFEE52080EEF6E65C0E9FF66C022
:1019D000EAFF020EE926000EEA22280EEE6E040E41
:1019E000ED6E63C0E9FF64C0EAFFEF50400B06E113
:1019F00065C0E9FF66C0EAFFC80E05D065C0E9FF13
:101A000066C0EAFF880EEF6E28D065C0E9FF66C0A9
:101A1000EAFFEE52080EEF6E65C0E9FF66C0EAFF0E
:101A2000020EE926000EEA22200EEE6E040EED6E86
:101A300065C0E9FF66C0EAFF840EEF6E7B517C1142
:101A400007E005D07CC0FAFF00017B51F96EFADF98
:101A50000001789F895101E1C6DD020EE15C02E2DE
:101A6000E16AE552E16EE552E7CFD9FF1200D9CF26
:101A7000E6FFE1CFD9FFE6520001738F010EE66E5B
:101A8000E66AE66A710EE66E0F0EE66E8AEC18F0F4
:101A90000B6E050EE15E0B50200EE66EE66AE66AFE
:101AA000000EE66E040EE66E8AEC18F00B6E050E64
:101AB000E15E0B506D8CDF6A020EDF5C10E2DF50DE
:101AC000EA6A840FE96E000EEA22EF6ADF50EA6AE2
:101AD000860FE96E000EEA22EF6ADF2AEDD7010ECB
:101AE000E66EE66AE66A620EE66E000EE66E8AEC66
:101AF00018F00B6E050EE15E0B506D9C0001080E98
:101B00006B6F040E6C6F000E636F040E646F63C026
:101B100065F0666F22C461F0615102E1100E12D0CF
:101B2000010EE66EE66A610EE66E000EE66E010ECE
:101B3000E66EE66A42EC17F00B6E060EE15E0B50A5
:101B40000001200E606FE552E552E7CFD9FF120089
:101B5000800E0401205D58E10001C00E736F040186
:101B60002351030A2FE0010A09E0030A4BE10001B7
:101B7000780E716F300E726F120E3ED02251F66EDB
:101B8000F76AD890F636F7360B0EF626310EF722A6
:101B90000900F5CF71F00A00F5CF72F0020E0001D6
:101BA000F76A7125F66E7251F7220800F5CF74F0CE
:101BB000030EF76A7125F66E7251F7220800F5CF11
:101BC00075F01200030E225D1AE22251F66EF76ADA
:101BD000D890F636F7360D0EF626310EF7220900AC
:101BE000F5CF71F00A00F5CF72F071C0F6FF72C048
:101BF000F7FF0800F5500001746F756B12000001CB
:101C0000736B12000001736B1200D9CFE6FFE1CFB6
:101C1000D9FF020EE1260401286B296B20511F0B0E
:101C2000020A11E0030A0CE0010A3CE10001738F93
:101C30000401288100017F0535E10401288332D0A9
:101C40000001738F2FD00001738F040124BF0BD0CC
:101C500024510F0BE96EEA6AD890E936EA36670E2E
:101C6000E926000E0AD024510F0BE96EEA6AD890DB
:101C7000E936EA366B0EE926000EEA22EECFDEFFE9
:101C8000EDCFDDFFDECFE9FFDDCFEAFFEF50800BC8
:101C900009E0DECFE9FFDDCFEAFFEF50040B02E001
:101CA000010E286F000173AF07D0280E716F040E6C
:101CB000726F7381020E746F020EE15C02E2E16AE0
:101CC000E552E16EE552E7CFD9FF120070A015D0C2
:101CD00063C0E9FF64C0EAFFEF5080080DE16BC00C
:101CE000E9FF6CC0EAFFEF50840806E163C0E9FF3A
:101CF00064C0EAFF8C0EEF6E7090689A12006984DF
:101D000068986D820001010E806F000EE66EE66A33
:101D1000E66EE66A750EE66EE66A42EC17F00B6E4A
:101D2000060EE15E0B5012000001806B000EE66EA5
:101D3000E66AE66EE66A740EE66EE66A42EC17F054
:101D40000B6E060EE15E0B506D92699468A402D092
:101D50006894FCD71200D9CFE6FFE1CFD9FFE65255
:101D600000012D0E886FFD0E811553E17E0E811549
:101D7000E8407F0B040DF3CF63F0F4CF64F0000E66
:101D80006327040E642363C065F064C066F0657564
:101D900063C0E9FF64C0EAFFEF503C0BE842E84251
:101DA0000D0835E1DF6A080EDF5C23E263C0E9FF5E
:101DB00064C0EAFF020EE926000EEA22EE50EFCFE1
:101DC000EAFFE96EEF50E66EDF50EA6A200FE96E37
:101DD000040EEA22E552E750EF6E63C0E9FF64C0EB
:101DE000EAFF020EE926000EEA22EE2AEF22DF2A9F
:101DF000DAD763C0E9FF64C0EAFF020EE926000EED
:101E0000EA22200EEE6E040EED6E0DD807D03AD801
:101E100005D0FD0E8115040801E159D8E552E552BF
:101E2000E7CFD9FF120000016F6B896B8C6B8D6B54
:101E3000836B706B6BC0E9FF6CC0EAFFEF9E6B7544
:101E40006BC0E9FF6CC0EAFFEF9E6B7565C0E9FFF0
:101E500066C0EAFFEF9E736B746B756B786B796B82
:101E60007A6B8CD8000EE66EE66AE66EE66A030EC2
:101E7000E66EE66A42EC17F00B6E060EE15E0B5062
:101E8000D8EF0BF0020E0001705D02E198EF0CF04C
:101E9000706B83511AE165C0E9FF66C0EAFFEE523C
:101EA000080EEF6E65C0E9FF66C0EAFF020EE92684
:101EB000000EEA22200EEE6E040EED6E65C0E9FF04
:101EC00066C0EAFF8C0EEF6E1200836B1200D9CF52
:101ED000E6FFE1CFD9FFE6526BC0E9FF6CC0EAFF35
:101EE000EF50400B01E0010EDF6E00016B75080E34
:101EF000605D08E122C46EFF6E5002E0100E01D05A
:101F0000040E606F700526E16BC0E9FF6CC0EAFF4C
:101F1000020EE926000EEA22280EEE6E040EED6E89
:101F2000A8DC020E00016F5D06E16BC0E9FF6CC02A
:101F3000EAFF840E0DD0DF5006E16BC0E9FF6CC0F4
:101F4000EAFFC80E05D06BC0E9FF6CC0EAFF880E3F
:101F5000EF6E0FD078AF0CD07B517C1107E005D02D
:101F60007CC0FAFF00017B51F96EFADF0001789F17
:101F7000706BE552E552E7CFD9FF12000401205102
:101F8000600BE842E842E842E842E842000901E02A
:101F9000120021510C0A50E00B0A3FE00C0A31E01C
:101FA000010A22E00B0A1EE0020A1CE0030A18E004
:101FB000080A10E0010A0CE00F0A08E0030A01E039
:101FC00012000001738F080E606F1200A8EF0DF071
:101FD00037EF0DF00001610E716F000E726F0CD0C3
:101FE00005EF0EF01DEF10F024510001716F726BC0
:101FF000620E7127000E72237381010E746F738F4E
:1020000012000001738F04012451EA6A620FE96E25
:10201000000EEA2222C4EFFF1200000EE66EE66A0E
:10202000E66EE66A020EE66EE66A42EC17F00B6EAA
:10203000060EE15E0B5012001200D9CFE6FFE1CF91
:10204000D9FF050EE1260401220510E120511F0BE6
:1020500000090CE10001738F030E0401215D04E10E
:102060000001010E7F6F02D000017F6B040122513D
:1020700001E011D120511F0B020801E00CD12451C5
:102080000F0B000901E107D124510F0B010801E2F8
:1020900002D1200E0001605D01E0FDD0738F0401CC
:1020A00024BF16D024510F0BE96EEA6AD890E936A6
:1020B000EA36670EE926000EEA22EECFDEFFEDCF0C
:1020C000DDFF24510F0BEA6A860FE96E000E15D072
:1020D00024510F0BE96EEA6AD890E936EA366B0EA6
:1020E000E926000EEA22EECFDEFFEDCFDDFF245120
:1020F0000F0BEA6A840FE96E000EEA22020EEFCFA0
:10210000DBFFD950020FE96EDACFEAFFEF50010B87
:1021100003E1000EDF9401D0DF8424BF0BD02451F3
:102120000F0BE96EEA6AD890E936EA36670EE926BF
:10213000000E0AD024510F0BE96EEA6AD890E936F6
:10214000EA366B0EE926000EEA22DECFEEFFDDCF87
:10215000EDFF030E215D20E1DECFE9FFDDCFEAFFD9
:10216000EF50800B11E024BF07D024510F0BEA6A17
:10217000860FE96E000E06D024510F0BEA6A840F19
:10218000E96E000EEA22EF82840EDECFE9FFDDCF9A
:10219000EAFFE850EF127FD0DF74DECFE9FFDDCF3A
:1021A000EAFFEF50800B1BE0DECFE9FFDDCFEAFF57
:1021B000EF9EDECFE9FFDDCFEAFFEF8C020EE66E89
:1021C000E66ADECFE6FFDDCFE6FF050EE66EE66AE5
:1021D00042EC17F00B6E060EE15E0B5005D0DECF21
:1021E000E9FFDDCFEAFFEF8CDF74D950020FE96E13
:1021F000DACFEAFFEF50020B07E1DECFE9FFDDCFD8
:10220000EAFFEF50800B2BE0040124BF07D02451DC
:102210000F0BEA6A860FE96E000E06D024510F0BF1
:10222000EA6A840FE96E000EEA22EF923B0E0B6E13
:10223000DECFE9FFDDCFEAFFE850EF16020EE66ED3
:10224000E66ADECFE6FFDDCFE6FF050EE66EE66A64
:1022500042EC17F00B6E060EE15E0B5007D03B0E02
:10226000DECFE9FFDDCFEAFFE850EF16040124518D
:102270000F0B0C6A700F0B6E0F0E0C22030E0BC0AF
:10228000DBFF040E0CC0DBFF030EDBCFE9FF040E07
:10229000DBCFEAFFEF90050EE15C02E2E16AE55276
:0A22A000E16EE552E7CFD9FF12000E
:0622AA00DACFE4FFE2CFF1
:1022B000DAFFE9CFE4FFEACFE4FFF6CFE4FFF7CFA0
:1022C000E4FFF5CFE4FFF3CFE4FFF4CFE4FFFACF70
:1022D000E4FF00EE00F00B0EE80403E3EECFE4FFB2
:1022E000FBD700EE0BF0030EE80403E3EECFE4FFB0
:1022F000FBD7E652AEEC08F09EAA10D0ABA20AD0F3
:102300000001AC6B00018E6B0001B1870001410E32
:10231000906F04D0AECF8EF00001B185E55200EE93
:102320000DF0030EE80403E3E5CFEDFFFBD700EE6D
:102330000AF00B0EE80403E3E5CFEDFFFBD7E5CF92
:10234000FAFFE5CFF4FFE5CFF3FFE5CFF5FFE5CFEB
:10235000F7FFE5CFF6FFE5CFEAFFE5CFE9FFE5CFF1
:10236000DAFF1100D8CFE4FFE0CFE4FFE46EDACF6C
:10237000E4FFE652F2A40AD0F2940A0E0001AE5D28
:1023800004E1AE6B0001B18101D0AE2BE552E5CF87
:10239000DAFFE550E5CFE0FFE5CFD8FF1000CEEC47
:1023A00015F0DCEC0AF00001B1830001B1A108D006
:1023B0008350800B02E08A8A01D08A9A0001B19191
:1023C0000001B1A503D032DB0001B1950001B1A934
:1023D0006ED09D9A0001B1BB60D00001AD51040ADE
:1023E00040E0070A2BE0010A16E0030A01E04CD0A6
:1023F000B4C0E6FFAFEC18F0E552B3C0E6FFAFECB7
:1024000018F0E55200018F510001B4250001B325F9
:1024100000018F6F41D0B6C0E6FFAFEC18F0E55277
:10242000B5C0E6FFAFEC18F0E55200018F51000196
:10243000B6250001B52500018F6F2ED0B8C0E6FF8C
:10244000AFEC18F0E552B7C0E6FFAFEC18F0E5527C
:1024500000018F510001B8250001B72500018F6FE1
:102460001BD0B9C0E6FFAFEC18F0E552B0C0E6FFF4
:10247000AFEC18F0E55200018F510001B9250001C1
:10248000B02500018F6F08D00001AC6B0001B1874F
:102490000001450E906F00D002D00001B1838FC0C3
:1024A000E6FFAFEC18F0E5529D8A0001B1990001FA
:1024B000B1A71FD09D9A450EE66EAFEC18F0E5521D
:1024C000720EE66EAFEC18F0E552720EE66EAFECEF
:1024D00018F0E552200EE66EAFEC18F0E55290C011
:1024E000E6FFAFEC18F0E552AB98AB889D8A00018F
:1024F000B1970001B1A303D07AD90001B1930400D0
:1025000083DB53D71200000191AF0BD00001AB5118
:102510000001D880A25503E20001B88F04D0A22B9D
:1025200002D00001A26B000191AD0BD00001AB51B4
:102530000001D880A15503E20001B88D04D0A12B81
:1025400002D00001A16B000191AB0BD00001AB5197
:102550000001D880A05503E20001B88B04D0A02B65
:1025600002D00001A06B000191A90BD00001AB517A
:102570000001D8809F5503E20001B88904D09F2B49
:1025800002D000019F6B000191A70BD00001AB515D
:102590000001D8809E5503E20001B88704D09E2B2D
:1025A00002D000019E6B000191A50BD00001AB5140
:1025B0000001D8809D5503E20001B88504D09D2B11
:1025C00002D000019D6B000191A30BD00001AB5123
:1025D0000001D8809C5503E20001B88304D09C2BF5
:1025E00002D000019C6B000191A10BD00001AB5106
:1025F0000001D8809B5503E20001B88104D09B2BD9
:1026000002D000019B6B000192AF0BD00001AB51D7
:102610000001D8809A5503E20001B78F04D09A2BAD
:1026200002D000019A6B000192AD0BD00001AB51BA
:102630000001D880995503E20001B78D04D0992B91
:1026400002D00001996B000192AB0BD00001AB519D
:102650000001D880985503E20001B78B04D0982B75
:1026600002D00001986B000192A90BD00001AB5180
:102670000001D880975503E20001B78904D0972B59
:1026800002D00001976B000192A70BD00001AB5163
:102690000001D880965503E20001B78704D0962B3D
:1026A00002D00001966B000192A50BD00001AB5146
:1026B0000001D880955503E20001B78504D0952B21
:1026C00002D00001956B000192A30BD00001AB5129
:1026D0000001D880945503E20001B78304D0942B05
:1026E00002D00001946B000192A10BD00001AB510C
:1026F0000001D880935503E20001B7811200932BAB
:1027000012000001936B12000001B8510001B413D4
:102710000001B7510001B31312008A92C69A8B8050
:102720008B82000000000000000000008A82000090
:1027300000000000000000008A920000000000007D
:1027400000000000C68A8B808B9200000000000011
:1027500000000000C96AC7A0FED7C9CF91F0C96ABE
:10276000C7A0FED7C9CF92F08B908B9200000000DB
:102770000000000000008A92C69A000000000000DD
:10278000000000008A82000000000000000000003D
:102790008A92C68A1200D9CFE6FFE1CFD9FFE6526E
:1027A000DF6A080EDF5C1CE28A92FE0EDB50800BB3
:1027B00002E0010E01D0000EE8B08A86E8A08A96F9
:1027C000FE0EDBCFF3FFF39EF346FE0EF3CFDBFFEF
:1027D0008A8200000000000000000000DF2AE1D72C
:1027E0008A928A96E552E552E7CFD9FF1200D9CFF7
:1027F000E6FFE1CFD9FF020EE126B9C0E6FFCBDF4D
:10280000E5520000B6C0E6FFC6DFE5520000B5C0E5
:10281000E6FFC1DFE5528B840000000000000000ED
:102820000000000000000000000000008B94000188
:10283000BAB102D08C9C01D08C8C0F0E0001AF1568
:10284000E8407F0BE76E010EE7CFDBFF010EDB50A8
:102850008D6EF00E0001AF15E8380F0B0A0A6FE01D
:10286000010A6DE0050A6BE0010A69E0060A5AE018
:10287000040A58E0050A49E0040A47E00A0A38E079
:10288000010A36E0020A2DE0010A24E0060A15E0FA
:10289000010A13E0020A0AE0010A01E05FD08C9805
:1028A0008C9A8C848C868C808C8258D08C988C8A64
:1028B0008C848C868C808C8251D08C988C9A8C8065
:1028C0008C820001AFB103D08C948C8602D08C84B2
:1028D0008C9644D08C888C9A8C848C868C808C824C
:1028E0003DD08C888C8A8C848C868C808C8236D06F
:1028F0008C988C9A8C848C860001AFB103D08C901C
:102900008C8202D08C808C9229D08C988C9A8C846A
:102910008C860001AFB103D08C908C8202D08C8069
:102920008C921CD08C988C8A8C848C860001AFB1E0
:1029300003D08C908C8202D08C808C920FD08C989B
:102940008C9A0001AFB105D08C948C868C908C82CF
:1029500004D08C848C968C808C9200D0010EDB503D
:10296000B9C0E7FF070B04E0E742E79EE806FCE199
:10297000E750010B1CE00001AFB10DD08C50010BF2
:1029800002E08C8201D08C928C50040B02E08C8689
:1029900001D08C960CD08C50020B02E08C8001D0C0
:1029A0008C908C50080B02E08C8401D08C94020E29
:1029B000E15C02E2E16AE552E16EE552E7CFD9FF60
:1029C0001200D9CFE6FFE1CFD9FFE652DF6AFE0E53
:1029D000DB380F0B070BE76EFE0EE7CFDBFFDB509C
:1029E000070A1BE0010A17E0030A13E0010A0FE0DF
:1029F000070A0BE0010A07E0030A03E0010A0FE1FE
:102A000004D0020E0BD0010E09D0DF6A08D0040EEC
:102A100005D00A0E03D0050E01D0060EDF6EDF389A
:102A2000F00BE552E552E7CFD9FF12000001AC519F
:102A3000050A01E175D0010A55E0070A35E0010AEF
:102A40000FE0030A08E0010A01E0A1D0550E0001E1
:102A50008E5D27E00ED0300E00018E5D0AE121D0A0
:102A60007F0E00018E1508E10001B1870001420EC2
:102A7000906F0001AC6B12007F0E8E150001AD6FE0
:102A8000860E00018E2500018F6F00018EBF07D0DA
:102A90000001B19B0001AC6B0001B1891200000183
:102AA000B18B0001AC2B1200AC2B00018F51000147
:102AB0008E2500018F6F0001AD51040A10E0070A56
:102AC0000BE0010A06E0030A01E012008EC0A3F049
:102AD00012008EC0A7F012008EC0A5F012008EC0AA
:102AE000A9F01200AC2B00018F5100018E250001CE
:102AF0008F6F0001AD51040A10E0070A0BE0010AD4
:102B000006E0030A01E012008EC0A4F012008EC09D
:102B1000A8F012008EC0A6F012008EC0AAF012001B
:102B200000018E5100018F5D2BE1A3C0B4F0A4C061
:102B3000B3F0A5C0B8F0A6C0B7F0A7C0B6F0A8C063
:102B4000B5F0A9C0B9F00001AA45010B0001BA6FA8
:102B5000AAC0B0F00F0E0001AA150B6EE66EAAC057
:102B6000E6FF2FDFE552E552E7CF0BF00B10000137
:102B7000AF6F0001AC6B00018F2B0001B189120017
:102B80000001AC6B0001B1870001430E05D0AC6BB6
:102B90000001B1870001460E906F12000F0EC112A6
:102BA00002D822EF08F0966A9398939A958E9490A3
:102BB00094929494959C9598959A959495969590C1
:102BC0009592939293969380948E949C8D6A8A8822
:102BD0008A9A8B908B928B948C9C8C988C9A8C94E8
:102BE0008C968C908C928A928A96C10ED56EF194B6
:102BF000F28AF28CA4EC18F00001C56BC66BC76BAF
:102C0000C86B010EC96F1200D9CFE6FFE1CFD9FF23
:102C1000E652200E0001E76E6019E8AE02D0E734FC
:102C200002D0E750605D01E2E1D06D50020B01E09F
:102C3000DDD00001C551C61102E1000E08D0C5C0AB
:102C4000E9FFC6C0EAFFEF50800B01E0010E00096A
:102C500001E0CCD005010051DB0A55E0DB0A09E0B8
:102C6000010A07E00001C751C81101E07FD0000E42
:102C700085D0000512E101C5B4F002C5B3F003C56B
:102C8000B6F004C5B5F005C5B8F006C5B7F007C580
:102C9000B9F008C5BAF009C5AFF00001C751C811B5
:102CA00002E1000E08D0C7C0E9FFC8C0EAFFEF503C
:102CB000800B01E0010E000901E085D000C540F560
:102CC000B4C041F5B3C042F5B6C043F5B5C044F554
:102CD000B8C045F5B7C046F5B9C047F5BAC048F524
:102CE000AFC049F50A0EDF6E400EDF5C09E2DF502F
:102CF000EA6A400FE96E050EEA22EF6ADF2AF4D78E
:102D00000001B1834DD00001C751C81102E1000E8E
:102D100008D0C7C0E9FFC8C0EAFFEF50800B01E050
:102D2000010E000950E100C540F50501010E416F9B
:102D3000020E426F030E436F040E446F050E456F83
:102D4000060E466F070E476F080E486F090E496F53
:102D50000A0EDF6E400EDF5C23E2DF50EA6A400FAE
:102D6000E96E050EEA22EF6ADF2AF4D7C7C0E9FF51
:102D7000C8C0EAFFEF50800B01E0010E000923E11B
:102D800005014069010EDF6E400EDF5C09E2DF5095
:102D9000EA6A400FE96E050EEA22EF6ADF2AF4D7ED
:102DA000400EE66E400EE66E050EE66E010EE66E15
:102DB000E66E98EC09F00B6E050EE15E0B50F3CF5A
:102DC000C7F0F4CFC8F0400EE66E000EE66E050EBA
:102DD000E66EE66A010EE66E98EC09F00B6E050EE3
:102DE000E15E0B50F3CFC5F0F4CFC6F0E552E552EB
:102DF000E7CFD9FF120012001200120012008CEF70
:102E000017F012001E0EE66E010EE66E61EC09F080
:102E1000E552E552400EE66E000EE66E050EE66ED9
:102E2000E66A010EE66E98EC09F00B6E050EE15EA7
:102E30000B50F3CFC5F0F4CFC6F0120000017F05B0
:102E400020E1000180051DE1A09AD6DF6D9200010E
:102E5000806B0001100ECC6F0E0ECD6FCC07000EF4
:102E6000CD5BCC51CD11FAE16D84080ECC6F070E0D
:102E7000CD6FCC07000ECD5BCC51CD11FAE16D9436
:102E8000A08A1200D9CFE6FFE1CFD9FFFD0EDBCF3C
:102E900006F0FE0EDBCF07F0050E061801E1075025
:102EA00036E0E868061802E17F0E07182FE0030EEF
:102EB000061801E1075028E0020E061801E107504C
:102EC00021E0010E061801E107501AE0740E061801
:102ED00001E1075013E0750E061801E107500CE000
:102EE000730E061801E1075005E0720E06180FE197
:102EF00007500DD082DF0BD07EDF09D07DDF07D0F9
:102F000081DF05D07EDF03D07ADF01D077DF010ECD
:082F1000E552E7CFD9FF1200E2
:082F1800040120511F0B010808
:102F200001E01200245101E01200060E215D1BE1B8
:102F30002351230A18E0010A0CE0030A14E10001FE
:102F4000610511E100019C0E716F300E726F090E68
:102F500006D00001EF0E716F300E726F1C0E746F91
:102F6000756BC00E736F04012051600BE842E8429C
:102F7000E842E842E842010801E0120021510B0A50
:102F800026E0080A19E0090A11E0080A05E00B0A20
:102F900023E0080A21E012000001CA0E716F000E42
:102FA000726F010E746F756BC10E0FD00001800E31
:102FB000736F23C4CAF012000001CB0E716F000EB4
:102FC000726F010E746F756B810E736F12000001CA
:0A2FD000800E736F22C4CBF01200D4
:062FDA002A0EF66E100E37
:102FE000F76E000EF86E00010900F550C06F090081
:102FF000F550C16F03E1C06701D03DD00900F55025
:10300000BB6F0900F550BC6F0900F550BD6F09009A
:103010000900F550E96E0900F550EA6E0900090053
:103020000900F550BE6F0900F550BF6F0900090097
:10303000F6CFC2F0F7CFC3F0F8CFC4F0BBC0F6FFB5
:10304000BCC0F7FFBDC0F8FF0001BE5302E1BF5393
:1030500007E00900F550EE6EBE07F8E2BF07F9D7AA
:10306000C2C0F6FFC3C0F7FFC4C0F8FF0001C0072D
:08307000000EC15BBFD7120086
:08307800120100020000000833
:10308000D8043F00020001020001090229000101E9
:1030900000C03209040000020300000009211101F0
:1030A0000001221C00070581034000010705010300
:1030B000400001040309041E03540075006C006104
:1030C00000700072006F006D007000720069006295
:1030D000006F0072001A034C0069006E0067006107
:1030E0000066006F006E00200033002E00300006E6
:1030F00000FF0901A10119012940150125407508AA
:1031000095408100190129409100C08A30B330B741
:0331100030D53087
:0C311400FE0EE3CFE9FFFF0EE3CFEAFF61
:10312000E9CFF3FFEACFF4FFFB0EE35003E1FC0E1F
:10313000E35009E0FB0EE30602E2FC0EE306FD0E9F
:08314000E350EE6EF1D712001E
:08314800B86A190EAF6EB06AFF
:10315000240EAC6E900EAB6E9F8A9D8A1200D9CF62
:10316000E6FFE1CFD9FF9EA8FED7FE0EDB50AD6E85
:08317000E552E7CFD9FF120080
:0831780013EE00F023EE00F05D
:10318000F86A0A9CEDEC17F0D1EC18F0CFEC11F0D6
:04319000FBD7120057
:0C31940000EE00F00F0EEE6AEA62FDD7BC
:0231A00012001B
:0231A200120019
:0531A400000000000125
:0731A900030000000000001C
:0931B00000000000000000000016
:020000040030CA
:0100000029D6
:010001000CF2
:010002003FBE
:010003001FDD
:010005008179
:010006008178
:010008000CEB
:01000900C036
:01000A000FE6
:01000B00E014
:01000C000FE4
:01000D0040B2
:00000001FF
